:020000000C28CA
:06000A0006280728082863
:1000100009280A280B28080085018601831610305C
:100020008500030186008F30810083128B018F01D0
:100030008E010301051A01308D00851485100D080D
:100040008C000301051A01308D000C0603191F28CE
:10005000051A2F2805202C28051E1F280000052022
:100060000000051A1F2805203528051E1F288F01AE
:1000700005200F11051A0F15052000008F10051A15
:100080008F14052000000F10051A0F148A018F0D20
:100090000F0D82070E1400008E1069280E1000004C
:1000A0008E1469280E1500008E1169280E110000AB
:1000B0008E1569280E1600008E1269280E12000097
:1000C0008E1669280E1700008E1369280E13000083
:0800D0008E170E08860021289E
:00000001FF
